:1000000012C0189518951895189518951895189563
:100010001895189518951895189518951895189578
:100020001895189518958FE58DBFC0E4E0E44E2E25
:1000300084E08EBFD4E0F4E05F2EEEEFF3E0A0E6C4
:10004000B0E0A89584B7082E877F84BF88E1992700
:1000500081BD91BD88278D933197E9F720D3662420
:100060008DEF87BB8CEF84BB8FEF81BB80E088BBBB
:10007000C19A80E085BB80E082BBE2E9F0E080E4E9
:1000800056D358E0C895802D4CD331965A95D1F768
:1000900004C010181C1E1E1C1810E2EBF0E088E4CF
:1000A00046D358E0C895802D3CD331965A95D1F768
:1000B00004C004040E0E0E1F1F1FE2EDF0E080E5E9
:1000C00036D358E0C895802D2CD331965A95D1F768
:1000D00004C01F1F1F0E0E0E040483E886B980E4BF
:1000E00087B98CE024D3C1D2E0E8FBE0B6D2BBD222
:1000F000E2E9FBE0B2D2E8E2F0E0ACE6B0E091E0A9
:1001000022D500916C000E3C08F00DC0AED2E0E8A4
:10011000FBE0A3D2A8D2E4EAFBE09FD285B78F7DB3
:10012000806A85BF889584E690E02DD380916C002D
:10013000815080936C00E8E2F0E0ACE6B0E091E042
:100140007BE7F0D4E2E0F0E0A1D2A0E6B0E0E6EB9D
:10015000FBE028D385E080936600ECE3F0E0AEE6B8
:10016000B0E091E0F0D4E2E3F0E0ADE6B0E091E0A1
:10017000EAD48FE711E088D2EAEBFBE06ED28FEB96
:1001800011E082D2EEEBFBE068D200916600053010
:1001900009F00AC08FE71BE077D281E0C2D28FEB73
:1001A0001BE072D282E0BDD280916E00809373001A
:1001B000EFD18FE711E068D2EAEBFBE04ED28FE798
:1001C00015E062D2FCD180916D0080937300E0D184
:1001D0008FEB11E059D2EEEBFBE03FD28FEB15E055
:1001E00053D2EDD1B998A0E7B0E09C9196FF04C03E
:1001F000B19B0EC09F7B9C93B1990AC088E29F93EC
:100200009927C1D29F91B19903C090649C934DD11D
:1002100000916600013009F048C0C598A0E6B0E042
:10022000E6EBFBE0BFD28FEB1EE02ED2A0E6B0E003
:100230000ED28FE71DE028D2E2ECFBE00ED280E088
:1002400080937400D4D1E4E7FBE0EDD3E7E6F0E07F
:10025000EBD25FD3EDE0F0E0B3D2AEE6B0E0DC92FB
:10026000AEE6B0E08C91845C8C9380916E008093BC
:1002700073008ED18FE715E007D2A1D1B998A0E71E
:10028000B0E09C9196FF04C0B19B0EC09F7B9C93F5
:10029000B1990AC088E29F93992775D29F91B1992D
:1002A00003C090649C9301D1B3CF009166000230EB
:1002B00009F048C0C598A0E6B0E0E6EBFBE072D2DA
:1002C0008FEB1EE0E1D1A0E6B0E0C1D18FE71DE0E9
:1002D000DBD1E2ECFBE0C1D180E08093740087D1F8
:1002E000E4E7FBE0A0D3E7E6F0E09ED212D3EDE036
:1002F000F0E066D2ADE6B0E0DC92ADE6B0E08C9125
:10030000865F8C9380916D008093730041D18FEB59
:1003100015E0BAD154D1B998A0E7B0E09C9196FF0E
:1003200004C0B19B0EC09F7B9C93B1990AC088E228
:100330009F93992728D29F91B19903C090649C9371
:10034000B4D0B3CF81E08093740051D1E8E7FBE0F3
:100350006AD3E7E6F0E068D232D3EDE0F0E030D2E5
:10036000AFE6B0E0DC9280916F008093730010D113
:100370008FE71DE089D1009171000A3008F003C0B9
:10038000E8ECFBE06AD1A8E2B4E0E1E7F0E071D389
:100390005CD1EAECFBE061D1A8E2B4E0E2E7F0E096
:1003A00068D353D100916600033009F01BC08091DF
:1003B0007000806880937000A0E6B0E0ECECFBE099
:1003C000F1D140916E0000916F00041708F40AC04B
:1003D000809170008F7780937000A0E6B0E0E6EB2C
:1003E000FBE0E0D100916600043009F01CC0809170
:1003F0007000806880937000A0E6B0E0ECECFBE059
:10040000D1D140916D0000916F00041710F009F0F8
:100410000AC0809170008F7780937000A0E6B0E0F2
:10042000E6EBFBE0BFD100916600053009F02DC07E
:1004300080917000806880937000A0E6B0E0ECECE2
:10044000FBE0B0D140916E0000916F00041708F4FA
:100450000AC0809170008F7780937000A0E6B0E0B2
:10046000E6EBFBE09FD140916D0000916F00041717
:1004700010F009F00AC0809170008F7780937000AF
:10048000A0E6B0E0E6EBFBE08DD1A0E7B0E08C9118
:1004900087FB0EF002C0C59A01C0C5988FEB1EE025
:1004A000F3D0A0E6B0E0D3D07FCEA6E6B0E08C914A
:1004B0008F5F8C9300916600053010F009F001C049
:1004C00003C081E08093660000916600013009F06E
:1004D00011C08FE71BE0D8D0E8ECFBE0BED08FEB7B
:1004E0001BE0D2D0E8ECFBE0B8D08FE714E0CCD032
:1004F00080E017D100916600023009F00BC08FEB4D
:1005000014E0C2D080E00DD18FE714E0BDD0E8EC5C
:10051000FBE0A3D000916600033009F019C08FE71B
:100520001BE0B2D081E0FDD08FEB14E0ADD0E8EC61
:10053000FBE093D0ECE3F0E0AEE6B0E091E07BE7E7
:10054000F1D2E2E3F0E0ADE6B0E091E07BE7EAD2A1
:1005500000916600043009F00BC08FE71BE094D0D7
:10056000E8ECFBE07AD08FEB1BE08ED082E0D9D0B4
:1005700000916600053009F00AC08FE71BE084D0C7
:1005800081E0CFD08FEB1BE07FD082E0CAD008950E
:10059000009173004AE0DED2A1E7B0E00C93009135
:1005A00071004AE0049FA2E7B0E00C920091730052
:1005B00040917200041BA2E7B0E00C9308950091F3
:1005C00071000A3008F003C0E8ECFBE046D0A8E276
:1005D000B4E0E1E7F0E04DD238D0EAECFBE03DD00A
:1005E000A8E2B4E0E2E7F0E044D22FD00895379AD1
:1005F000EF93FF93E5E1F0E0BAD0FF91EF9107B1FF
:10060000007FA4E7B0E08C9190E0890F082707B93C
:10061000CED0A4E6B0E08D939C933798E4E6F0E06A
:10062000D190E080FF24002723D1A7E6B0E051D18C
:10063000ECE7FBE0F8D1E7E6F0E0F6D0C0D1EDE082
:10064000F0E0A7E6B0E05FD20895A8E2B4E08D91B3
:10065000882311F066D0FBCF0895E1D1802D11F0F1
:1006600060D0FBCF089580EC62C081E060D014D0F0
:1006700080E85DC08FE7213039F08FEB223021F028
:100680008FE8233009F08FEC810F51C088EE93E0A2
:100690007AD03197D9F7089583E0992774C08AEF0B
:1006A00090E071D0A59AA49AA39AA29A889A899A5E
:1006B000919885E090E067D09098AD98AC98AB9A0F
:1006C000AA9A909AEF93FF93E5E1F0E050D0FF9162
:1006D000EF91909855D0909AEF93FF93E5E1F0E079
:1006E00046D0FF91EF9190984BD0909AEF93FF9363
:1006F000E5E1F0E03CD0FF91EF91909841D0AA98CD
:10070000909AEF93FF93E5E1F0E031D0FF91EF9104
:10071000909836D088E20BD08EE009D086E007D0E2
:100720000895919A829505D004D02AD00895919881
:10073000F9CF859510F4AA9A01C0AA98859510F46E
:10074000AB9A01C0AB98859510F4AC9A01C0AC98F7
:10075000859510F4AD9A01C0AD98909AEF93FF93F0
:10076000E5E1F0E004D0FF91EF9190980895319782
:10077000F1F70895689462F80895E89462F808958E
:1007800081E090E000C0EF93FF93EE27E82BE92B88
:1007900031F0EAEFF0E03197F1F70197D1F7FF91EF
:1007A000EF9108953CD10D920020E1F70895369A1B
:1007B0003699FECF369A3699FECF84B195B1089519
:1007C00033D0992711278F2D880F80E8F82A802FA2
:1007D000881F08F41FEF41F08F57082F07FD04C052
:1007E000003240F08FEF01C08827982FD82EE82ED6
:1007F000F82E09C08FE1801B082FF694E794D79458
:1008000097950A95D1F7112351F09095D094E094E3
:10081000F09481E0980F8827D81EE81EF81E0F2D4F
:10082000FE2CED2CD92E0895D190E190F1900191FC
:10083000089521913191419151910895102F90E89F
:10084000FF0C001F0927990FF7941078652F90E887
:10085000440F551F5927990F479560780038089520
:10086000FF0C90E89027110F9795F794092F0895A2
:10087000102FBD2CDE2CEF2CF02E11234AF4B09457
:10088000D094E094F0949FEFB91AD90AE90AF90AD2
:100890000EE1FF2039F4FE2CED2CDB2CBB2408509C
:1008A000C2F76BC032F00A95BB0CDD1CEE1CFF1CBE
:1008B000F9CF01D0D5CFB7FE089590E8B91611F45D
:1008C000D0FE08959FEFD91AE90AF90A09F40395B1
:1008D0000895DD92ED92FD920C930895502F2D2DE9
:1008E0003E2D4F2D612F08952DEC3CEC4CEC5DE33B
:1008F00066270FC099DFF2DFDD24EE2490E8F92EA1
:100900000FE307C096DF05C02227332740E251E4FA
:100910006627552351F1002381F190DF71F11627ED
:10092000005850580894050B18F407FD03C025C063
:1009300007FD23C0469537952795F694E794D794FD
:1009400022D0FF202AF0DD0CEE1CFF1C015073F0BA
:100950009D2D969548F0DD203AF4EE202AF491E0A2
:10096000D90E9927E91EF91E7BCF07C09FE7092FF3
:10097000F92A9FEFD92EE92E0895DD24EE24FF24D5
:100980000027112708959F929924AA24BB2488E167
:10099000D216E306F40628F0D21AE30AF40A089401
:1009A00001C08894991CAA1CBB1CDD0CEE1CFF1C0A
:1009B0008A9571F7D92CEA2CFB2C9F9008953EDF85
:1009C000E1F25038D1F21627005850580894051F0C
:1009D00012F418F4CBCF08F0D0CF0AD0FF202AF0C1
:1009E000BB0CDD1CEE1CFF1C3BCF0F5FFBF138CFB7
:1009F0009F929924AA24BB24992788E1990CAA1CC8
:100A0000BB1CDD1CEE1CFF1C30F4920EA31EB41E9A
:100A1000D91EE91EF91E8A9589F79F900895C895F9
:100A2000319600200895FBDF202DF9DF302DF7DF10
:100A3000402DF5DF502D0895000F111F221F331F89
:100A4000089500951095209530950F5F1F4F2F4FFB
:100A50003F4F0895019110810EC001911191219194
:100A600030810BC00191108117FF05C03FEF2FEFC0
:100A700004C0008111272227332737FF03C0E1DF9D
:100A80008DE28D93CF93DF93CF92DF92EF92AA24E2
:100A9000BB24CC24DD24EE2440E2CAE0DD2755E06F
:100AA00093E38881890F87FD9F7083FD907F891B69
:100AB00089935A95A9F7C0DFAA1CBB1CCC1CDD1C6E
:100AC000EE1C4A9551F7E894EFE0FF2782910ED093
:100AD000EB30E0F71EF068948A2D0CD088278D93B8
:100AE000EF90DF90CF90DF91CF910895982F82956E
:100AF00001D0892F8F70805D26F0803309F408952E
:100B000068948D93089594E081918D939A95E1F77F
:100B10000895E199FECFEEBBFFBB3196089591E0B9
:100B200001C092E07B3751F47FB7F894F2DF8D91EA
:100B30008DBBE29AE19A9A95C9F77FBF772708950E
:100B400091E001C092E0E5DFE09A8DB38D939A9534
:100B5000D1F70895FF93881BF9E0001FFA9511F46F
:100B6000FF910895881F841B18F4840F8894F5CF93
:100B70000894F3CF0000A040F628DC3E23DBF93ECA
:100B80005757572E4156522E344D472E434F4D2026
:100B90000000414B5520636F6E74726F6C205631AC
:100BA0002E32000054484520454E44204F462044F4
:100BB000454D4F2100004F46460055323D0055310E
:100BC0003D0020202020000020002E004F4E20005D
:00000001FF
